:0200000480007A
:100000006F008004732F2034930F80006308FF0378
:10001000930F90006304FF03930FB0006300FF038E
:10002000130F000063040F0067000F00732F2034CC
:1000300063540F006F00400093E19153171F0000BD
:1000400023223FFC6FF09FFF93000000130100008C
:10005000930100001302000093020000130300004C
:100060009303000013040000930400001305000034
:10007000930500001306000093060000130700001C
:100080009307000013080000930800001309000004
:1000900093090000130A0000930A0000130B0000EC
:1000A000930B0000130C0000930C0000130D0000D4
:1000B000930D0000130E0000930E0000130F0000BC
:1000C000930F0000732540F16310050097020000B4
:1000D000938202017390523073500018970200000F
:1000E00093824202739052309B021000939252030B
:1000F0009382F2FF7390023B9302F0017390023AF5
:100100007350403097020000938242017390523046
:10011000735020307350303093010000970200007C
:10012000938282EE73905230130510001315F5017F
:10013000635C05000F00F00F930110009308D005D9
:10014000130500007300000093020000638A0200A0
:1001500073905210B7B200009B82921073902230BD
:100160007350003097020000938242017390123462
:10017000732540F17300203097200000938080E8C1
:1001800003A70000B703FF009B83F30F9301200038
:10019000631A7726972000009380C0E603A74000EB
:1001A000B70301FF9B8303F093013000631C7724A6
:1001B00097200000938000E503A78000B713F00F9D
:1001C0009B8303FF93014000631E7722972000006A
:1001D000938040E303A7C000B7F30FF09B83F300C5
:1001E000930150006310772297200000938040E233
:1001F00003A740FFB703FF009B83F30F9301600049
:100200006312772097200000938080E003A780FF8F
:10021000B70301FF9B8303F0930170006314771E03
:10022000972000009380C0DE03A7C0FFB713F00F34
:100230009B8303FF930180006316771C97200000C7
:10024000938000DD03A70000B7F30FF09B83F3005A
:10025000930190006318771A97200000938080DA4A
:10026000938000FE83A20002B703FF009B83F30F7D
:100270009301A0006398721897200000938080D8A3
:100280009380D0FF83A27000B70301FF9B8303F02C
:100290009301B000639872169301C000130200002E
:1002A00097200000938040D603A740001303070067
:1002B000B713F00F9B8303FF63167314130212002E
:1002C00093022000E31E52FC9301D00013020000B1
:1002D00097200000938080D303A740001300000004
:1002E00013030700B7F30FF09B83F300631C731035
:1002F0001302120093022000E31C52FC9301E00061
:1003000013020000972000009380C0CF03A7400095
:10031000130000001300000013030700B70301FFE0
:100320009B8303F06310730E1302120093022000EC
:10033000E31A52FC9301F000130200009720000022
:10034000938080CC03A74000B713F00F9B8303FF7B
:10035000631A770A1302120093022000E31052FE80
:10036000930100011302000097200000938000CA4F
:100370001300000003A74000B7F30FF09B83F300C6
:10038000631277081302120093022000E31E52FC4E
:10039000930110011302000097200000938080C693
:1003A000130000001300000003A74000B70301FF83
:1003B0009B8303F06318770413021200930220005A
:1003C000E31C52FC972200009382C2C303A10200E7
:1003D0001301200093032000930120016314710294
:1003E00097220000938202C203A1020013000000C2
:1003F0001301200093032000930130016314710066
:10040000631030020F00F00F638001009391110020
:1004100093E111009308D0051385010073000000DB
:100420000F00F00F930110009308D0051305000092
:0C04300073000000731000C0000000000A
:1010000000000000000000000000000000000000E0
:1010100000000000000000000000000000000000D0
:1010200000000000000000000000000000000000C0
:1010300000000000000000000000000000000000B0
:081040000000000000000000A8
:10200000FF00FF0000FF00FFF00FF00F0FF00FF0D8
:040000058000000077
:00000001FF
